:020000040800F2
:1000000000020020A1040008B1130008B513000885
:10001000F1130008B5130008D1130008A304000869
:10002000A3040008A3040008A3040008213000086A
:10003000A3040008A3040008A304000895350008E1
:10004000A3040008A3040008A3040008A3040008F4
:10005000A3040008A304000899320008C532000870
:10006000F13200081D33000849330008A3040008DA
:10007000A3040008A3040008A3040008A3040008C4
:10008000A3040008A3040008A30400080525000831
:1000900071250008C52500081926000875330008D9
:1000A000A3040008A3040008A3040008A304000894
:1000B000A3040008A3040008A3040008A304000884
:1000C000A3040008A3040008A3040008A304000874
:1000D000A3040008A3040008093700081D3700081E
:1000E000DD330008A3040008A3040008A3040008EB
:1000F000A3040008A3040008A3040008A304000844
:10010000A3040008A3040008A3040008A304000833
:10011000A3040008A3040008A3040008A304000823
:10012000A3040008A3040008A3040008A304000813
:10013000A3040008A3040008A3040008A304000803
:10014000A3040008A3040008A3040008A3040008F3
:10015000A3040008A3040008A3040008A3040008E3
:10016000D0400B1CD1409C46203AD3401843524209
:1001700063469340184370479140031C90409C464F
:10018000203A9340194352426346D3401943704783
:1001900053B94AB9002908BF00281CBF4FF0FF31EE
:1001A0004FF0FF3000F07AB9ADF1080C6DE904CEE4
:1001B00000F006F8DDF804E0DDE9022304B0704742
:1001C0002DE9F0478C460E460446089D002B50D181
:1001D0008A4217466CD9B2FA82FEBEF1000F0BD0EC
:1001E000CEF1200C01FA0EF620FA0CFC02FA0EF702
:1001F0004CEA060C00FA0EF43A0CBCFBF2F9BBB266
:1002000002FB19CC09FB03FA4FEA144848EA0C46F2
:10021000B2450AD9F61909F1FF3180F02581B245BE
:1002200040F22281A9F102093E44A6EB0A06B6FB80
:10023000F2F002FB106600FB03F3A4B244EA0644AA
:10024000A34209D9E41900F1FF3280F00B81A342E7
:1002500040F2088102383C440021E41A40EA094097
:10026000002D62D0002324FA0EF42C606B60BDE8F0
:10027000F0878B4207D9002D55D0002185E8410039
:100280000846BDE8F087B3FA83F1002940F08F807B
:10029000B34202D3824200F2FC80841A66EB03066A
:1002A0000120B446002D40D085E81010BDE8F0874D
:1002B00012B90127B7FBF2F7B7FA87FEBEF1000FBC
:1002C00035D10121F61B4FEA174C1FFA87F8B6FB10
:1002D000FCF20CFB126608FB02F0230C43EA064614
:1002E000B04207D9F61902F1FF3302D2B04200F250
:1002F000D2801A46361AB6FBFCF00CFB106608FBDF
:1003000000F8A3B243EA0644A04507D9E41900F176
:10031000FF3302D2A04500F2B9801846A4EB0804CE
:1003200040EA02409CE729462846BDE8F08707FAE4
:100330000EF7CEF1200326FA03F24FEA174CB2FB78
:10034000FCF11FFA87F80CFB112206FA0EF620FAD0
:1003500003F301FB08F933431E0C46EA0246B1459C
:1003600000FA0EF409D9F61901F1FF3280F08C8001
:10037000B14540F2898002393E44A6EB0906B6FB3E
:10038000FCF00CFB106200FB08F99EB246EA024644
:10039000B14507D9F61900F1FF3371D2B1456FD9D4
:1003A00002383E44A6EB090640EA01418FE7C1F15D
:1003B000200722FA07F88B4048EA030326FA07F4DD
:1003C0004FEA134EB4FBFEF91FFA83FC0EFB1944EF
:1003D0008E4020FA07F809FB0CFA48EA06084FEAB3
:1003E000184646EA0444A24502FA01F200FA01F670
:1003F00008D9E41809F1FF3044D2A24542D9A9F145
:1004000002091C44A4EB0A04B4FBFEF00EFB1044EA
:1004100000FB0CFC1FFA88F848EA0444A44507D9FD
:10042000E41800F1FF3E29D2A44527D902381C4424
:1004300040EA0940A0FB0289A4EB0C0CCC45C24663
:10044000CE4615D312D055B1B6EB0A036CEB0E06AF
:1004500006FA07F7CB401F43CE402F606E600021A5
:10046000BDE8F0871046F7E68946DEE64645EAD263
:10047000B8EB020A69EB030E0138E4E77046D7E7F0
:1004800018468FE78146BDE7114676E702383C44BF
:1004900044E7084606E7023A3E442BE7704700BFB0
:1004A00002E000F000F8FEE772B6274880F3088803
:1004B000264880F3098826484EF60851CEF20001FE
:1004C0000860022080F31488BFF36F8F02F0D8FD1C
:1004D00002F070FE4FF055301E491B4A91423CBF5E
:1004E00041F8040BFAE71C49184A91423CBF41F815
:1004F000040BFAE719491A4A1A4B9A423EBF51F8BF
:10050000040B42F8040BF8E700201749174A914200
:100510003CBF41F8040BFAE702F0B6FD02F04CFED6
:10052000134C144DAC4203DA54F8041B8847F9E726
:1005300000F03AF8104C114DAC4203DA54F8041BA9
:100540008847F9E702F09EBD000200200008002065
:1005500000000008000100200002002038410008CF
:10056000000800207808002078080020542400208B
:1005700060010008600100086001000860010008D7
:100580002DE9F04FC1F80CD0C3689D46BDE8F08F4F
:10059000002383F311882846A047002002F036FB91
:1005A00002F0DCFA00DFFEE76FF01202F8B53E4B16
:1005B00000241A70032270215A709A723B4A5972B1
:1005C0009C70DC701C715C719C71DC711C72DC7243
:1005D000536823F0E06343F0905343F48043536047
:1005E00002F0C8FC074602F015FD0646A0BB304BE2
:1005F0009F4233D001339F4233D02E4B27F0FF026E
:100600009A4231D1F8B200F059FA354642F21074EC
:1006100000F08AFC00F058FA88B34CBB2EB1264B90
:100620009F4202D002F0EEFC0025002002F0ACFC5C
:1006300015B1002500F042F800F098FC00F032FE01
:1006400000F0E4FE044605B300F0E0FE001BA84203
:100650001BD900F033F8F3E70546D9E70546044611
:10066000D6E704460125D3E7054641F28834CFE7B3
:10067000AEB9002002F088FC4FF47A75DAE756B97B
:10068000002002F081FC0025D6E700F0C5FC012027
:1006900002F0C2FAD7E7084B9F42C3D1F0E7064BFE
:1006A0009F42BFD1E5E700BF78080020000001406D
:1006B000010007B0000008B0263A09B010B51C4B85
:1006C0001C4953F8042F013200D110BD8B42F8D1E0
:1006D000194C1A4B22689A4228D9194B9B6803F18E
:1006E000006303F508439A4220D202F05FFC02F057
:1006F00071FC002000F0FCFD0220124B187000F08D
:100700002BFE114BDA690022DA61D96999699A6185
:100710009B6972B60D4B0E4A202113601B6822683C
:1007200081F311889D4683F30888104710BD00BFF0
:10073000FC8700081C88000804880008FF87000860
:10074000780800208408002000100240008800087B
:1007500008ED00E049F2690008490B689AB21B0CE9
:1007600000FB02330B6044F25061054A136898B2F3
:100770001B0C01FB0030106080B270471008002095
:100780000C08002010B504460021102200F000FEE5
:10079000034B03CB206061601868A06010BD00BFF0
:1007A000E8F7FF1FF0B5BBB000F030FE1D4CA368AA
:1007B000C31AF92B30D906AD2346A06028220021A8
:1007C000284601F0B1FB04F10E0000F0D9FD002332
:1007D000C6B2591D5F1CDBB2B3424FEAC10107DA52
:1007E0000E3323440822284601F09EFB3B46F0E7E7
:1007F00001230393082302930B4B207B01933023A7
:10080000C1F3CF0105910093014604A3D3E900236E
:100810000495064801F058F93BB0F0BD78F6339FD7
:1008200093CACD8DC8180020D5180020A01800202C
:1008300070B50D4614461E4601F0ECF850B9022E74
:100840000ED1012C0CD112A3D3E90023C5E900235A
:10085000012070BD052C14D003D8012C09D0002034
:1008600070BD282C09D0302CF9D10BA3D3E900237B
:10087000ECE70BA3D3E90023E8E70BA3D3E90023BC
:10088000E4E70BA3D3E90023E0E700BFAFF3008068
:10089000401DA12026812A0B78F6339F93CACD8D67
:1008A0009E6AC421818A46EE26417272DF25D7B73F
:1008B000F017304A39059E5638B50D4604460346B2
:1008C00020222846002101F02FFB22792346032A0B
:1008D00028BF0322284603F8042F2021022201F01A
:1008E00023FB62792346072A28BF0722284603F8FC
:1008F000052F2221032201F017FBA2792346072AA4
:1009000028BF0722284603F8062F2521032201F0DD
:100910000BFB284604F108031022282101F004FBF8
:10092000382038BD2DE9F04FADF5037D23AE10AD75
:1009300040F2791280460F463046002100F028FD33
:1009400048220021284600F023FD00F05FFD4FF40F
:100950007A72B0FBF2F0574B0DF16209186093E820
:10096000070001232B74002385E807000DF16200C6
:100970006B74FFF707FF032385F82030ED2385F81C
:10098000213007AB18464C4903F09CF8212228641B
:100990003146284685F83C20FFF78EFF14AB04460D
:1009A00001460822304601F0BFFA08220DF151033A
:1009B000A118304601F0B8FA0DF15203082204F1F3
:1009C0001001304601F0B0FA15AB202204F11801F5
:1009D000304601F0A9FA16AB402204F13801304646
:1009E00001F0A2FA18AB082204F17801304601F0B8
:1009F0009BFA0DF16103082204F18001304601F0F9
:100A000093FA04F1880A04F5847B4B465146082288
:100A100030460AF1080A01F087FAD34509F10109C5
:100A2000F3D11DAB08225946304601F07DFA4FF054
:100A3000000904F5887495F834304B4510D84FF010
:100A4000000995F83C304B4515D92B6C21464B4499
:100A50000822304601F068FA083409F10109F0E78C
:100A6000AB6B21464B440822304601F05DFA083456
:100A700009F10109DFE7E31DC3F3CF03F97E059315
:100A8000002304960393BB7E193702930123019739
:100A90000093404605A3D3E9002301F015F80DF5B6
:100AA000037DBDE8F08F00BFAFF300809E6AC421D4
:100AB000818A46EE880800207C3C0008014B1870B3
:100AC000704700BF94080020F0B52E4B85B01C7B0A
:100AD0002CB10E222C4B1A81002005B0F0BD2B4A00
:100AE00002AB1068516803C3082329490DEB0302C8
:100AF000284802F0C9FF054630B90A22224B264891
:100B00001A8100F04DFCE7E70369B3F55E3F07D9B2
:100B10000B211D4A21481181194600F041FCDBE7F9
:100B200040F2ED32418B914206D00C20164B1881D9
:100B30001B4800F035FCCFE71A4A103B0244154928
:100B400020469E1A00F066FC0746324605F1180161
:100B5000204600F05FFCAB689F4202D1EB689842F0
:100B60000AD00D22084B1A8100903B46EA68A9681A
:100B70000D4800F015FCAFE70C4800F011FC012017
:100B8000ABE700BFC8180020880800206C3B0008B5
:100B9000DC77030000880008743B0008803B0008F5
:100BA000923B00080878FFF7B03B0008D93B0008EB
:100BB0002DE9F04FAFB006AF80460D4600F02AFF9A
:100BC000044600286CD12B7E022B18D1EB8A012B16
:100BD00015D100F01BFC8146FFF7BCFD4FF4C87334
:100BE000B0FBF3F202FB1300BD4E80B209F516799B
:100BF000EB7E4844306093B90022BA4B1A70A43798
:100C0000BD46BDE8F08F07F10C031C44009400239F
:100C100008224FEAC901284600F0EAFF4C46AB8A99
:100C20005FFA84F9013BA3420BD904F10109B9F140
:100C3000110FE8D140F23911AB4BAC4AAC4802F08D
:100C4000F5FE07F11C00FFF79DFD224607F11C0190
:100C500007F10C0002F008FF03460028CCD1B9F1DF
:100C6000100F07D09F4B83F800903368A3F51673DD
:100C70003360C4E707F1A00202F8950D0146009227
:100C80002846072200F0B4FFF97A7F2904DD994B4A
:100C9000964A4FF4A871D1E7404600F09FFEAEE7B8
:100CA000EB8A052B00F02E8106D8012BA7D129460F
:100CB0004046FFF737FEA2E7282B3DD0302B9ED1D0
:100CC0006B7E8D4C0133627BDBB29342EA4640F08F
:100CD0000081EA7E237B9A4240F0FB80002607F1E8
:100CE000A00323F8846D0093102201233146284687
:100CF00000F07EFFB5F81480A8F102081FFA88F80A
:100D000008F1030323F003030A3323F00703ADEBD9
:100D1000030D0DF1180933469BB2B11C98454FEAFB
:100D2000C10106F101066DDD4B440093082200234A
:100D3000284600F05DFFEEE7AB8A013B9BB2C92B72
:100D40003FF65DAF6C4E347B4CBB06F10C03009359
:100D5000082223462146284600F04AFFAB8A04F1C8
:100D60000109013BE4B29C424FEAC90109DA0E34A1
:100D70003444009400230822284600F039FF4C46F2
:100D8000ECE700230022C6E900230023B36086F8C5
:100D9000D730C6F8D830337B0BB9EB7E33730024E1
:100DA00007F11C0607F10C03082221463046FC60BF
:100DB0003C617C6101F0B8F83B7C04F10109A3427D
:100DC0004FEAC90107D97B6908222344304601F064
:100DD000ABF84C46F0E70023C1F3CF01E87E059164
:100DE00004960393AB7E19350293282301460093A2
:100DF000019539A3D3E90023404600F065FEFFF7D3
:100E0000D1FCFCE694F8D70000F084FAD4F8D8308E
:100E100006461BB994F8D70000F08CFAD4F8D83005
:100E200043449E4204D294F8D700013000F082FA85
:100E30000025324B4FEA980BAAB25A45104616DAF3
:100E40005AB994F8D72042B9D4E900120A4304D120
:100E5000D9F800201A600135EEE7226859F8201011
:100E600002EB80007B6000F045FA7B68F3E7D4E991
:100E70000023D4F8D85012EB080043F10001C4E974
:100E80000001454494F8D700C4F8D85000F042FA65
:100E9000854209D394F8D730013384F8D730D4F899
:100EA000D8309E1BC4F8D860B8F1FF0F0ADC0020D0
:100EB000124B2073196800F01DFAFFF705FE08B108
:100EC000FFF7FCFB23680E4A9B0A013313810023C2
:100ED000A360D54693E600BF26417272DF25D7B7DF
:100EE0009C18002099180020E83B0008A03C00084E
:100EF000413C0008633C0008C8180020000800209E
:100F000088080020BFF34F8F0549064BCA6802F4DA
:100F1000E0621343CB60BFF34F8F00BFFDE700BF1C
:100F200000ED00E00400FA0508B54FF000530B4A4D
:100F3000196891420AD1597D094A0A4811701B7DEE
:100F4000C922037308490E3000F010FABDE80840CA
:100F5000E02200214FF0005000F01ABA9AAD44C5CB
:100F600094080020C818002016000020022330B585
:100F70001F4C85B0637104230025ADF808300123B0
:100F80000722ADF80C501B498DF80C308DF80B3052
:100F9000194B1A484B608DF80A2001F0E5FC184BFC
:100FA000019500931749184B4FF48052174800F0F1
:100FB000DFFC174B2546197811B1144800F00EFDDF
:100FC00000F024FA0446FFF7C5FB4FF4C873B0FBEA
:100FD000F3F202FB130304F516749BB21C440D4B91
:100FE0001C6002F017F808B10F232B8105B030BD4B
:100FF000880800200408002003000600B81900201B
:101000003108000898080020B10B0008A018002043
:10101000940800209C1800202DE9F04F96A7D7E9EE
:1010200000670FF25C29D9E900898F4C93B0DFF893
:1010300058B2DFF858A2204600F092FD0CAD0790A0
:1010400098B310220021284600F0A2F94FF00002C8
:10105000079B197B61F3030219468DF8302051F884
:10106000040F0EAA496803C21B680D9A584663F321
:101070001C029DF830300D9243F020038DF8303083
:1010800000232A46194601F07FFC079030B920461C
:1010900000F06AFD079B8AF80030CCE79AF8003030
:1010A000072B40DC01338AF8003018220021284643
:1010B00000F06EF9DFF8D0B1DFF8D4A100232A46A2
:1010C0001946584601F088FC014680BB102208A84A
:1010D00000F05EF9DAF80C3083F00803CAF80C303F
:1010E00000F096F90DF1240E0B4612A9024611E903
:1010F00003008EE803009DF83410C1F30300890655
:1011000049BF0E99BDF83810C1F31C0141F00041F0
:1011100058BFC1F30A018DF82C000891204608A998
:1011200000F068FFCAE7204600F01EFDBDE720463C
:1011300000F070FC824600284AD100F067F9DFF821
:1011400054B1DBF80030984242D300F05FF90790C9
:10115000FFF700FB4FF4C873B0FBF3F101FB130082
:10116000079A80B202F516721044CBF80000DFF83F
:1011700028B18DF820A09BF8001011B901238DF83B
:10118000203028460791FFF7FDFA07990DF121005D
:10119000C1F1100A5FFA8AFABAF1060F28BF4FF0C0
:1011A000060A2944524600F0E1F80AF101030493CB
:1011B00008AB0393182302932C4B3246019301236F
:1011C000204600933B4600F027FC00238BF80030BC
:1011D00000F01CF9264ADFF8C4A01368C31AB3F55F
:1011E0007A7F32D3106000F013F902460B46204696
:1011F00000F0C0FC204600F00DFC30B39AF80C3033
:10120000DFF89CB0002B14BF032302238BF80530BA
:1012100000F0FCF84FF47A73B0FBF3F02946CBF8FA
:1012200000005846FFF748FB18230293114B073084
:10123000019340F25513C0F3CF000490009303953F
:1012400042464B46204600F0E7FB9AF80C300BB1C3
:10125000FFF7A8FA9AF80C30002B7FF4E8AE13B031
:10126000BDE8F08FAFF30080A01800209818002090
:10127000A8190020AC190020401DA12026812A0BAE
:10128000F1C6A7C1D068080FB8190020AD19002019
:10129000000C01409C18002099180020C81800205C
:1012A0008808002070B501F06DFD00250E4C0F4E32
:1012B00020703068237883420CD8002520780138CC
:1012C00001F05CFD23780544013BB5F5006F237008
:1012D000F4D370BD01F052FD336805440133B5F518
:1012E000084F3360E5D3E8E7B4190020B0190020B7
:1012F00001F0D6BD07B502AB43F8041D00F1006054
:101300000422194600F5084001F076FD03B05DF8AF
:1013100004FB0000054B1A68054B1B789B1A83429F
:1013200002D9104401F02ABD00207047B0190020F6
:10133000B419002038B50446064D2868204401F051
:1013400023FD28B928682044BDE8384001F02EBDAF
:1013500038BD00BFB0190020022802BF4FF40022A0
:10136000014B1A61704700BF000C0140002310B50B
:10137000934203D0CC5CC4540133F9E710BD0000A4
:1013800002460346981A13F9011B0029FAD1704747
:1013900003460244934202D003F8011BFAE7704768
:1013A0000FB4002004B070470EB4002003B07047A3
:1013B000FEE70000EFF30983EFF30583034B9A6B1D
:1013C0009A6A9A6A9A6A9A6A9B6AFEE700ED00E056
:1013D000EFF30983EFF30583044B9A6B9A6A9A6AD9
:1013E0009A6A9A6A9A6A9B6AFEE700BF00ED00E07B
:1013F000EFF30983EFF30583034B5A6B9A6A9A6AFA
:101400009A6A9A6A9B6AFEE700ED00E001F080BDEF
:1014100001F05ABD30B5084D0A4491420BD0092461
:1014200011F8013B5840013CF7D040F300032B403A
:1014300083EA5000F7E730BD2083B8ED024600682C
:1014400048B1036811891360D38801339BB2994274
:10145000D38038BF1381704770B504460D4688B0FD
:10146000202200216846FFF793FF20460495FFF7EE
:10147000E5FF054658B16B46044608AE1A4603CA56
:10148000B24220606160134604F10804F6D1284698
:1014900008B070BD2DE9F04130B940F2C531264B9E
:1014A000264A274802F0C2FA0B7C23B9254B234A6F
:1014B00040F2C631F5E7C66986B9C161BDE8F08181
:1014C000002B29DA930CAB4229D1B44201D10C6034
:1014D000F3E7C8F800100C60BDE8F0814B68B04637
:1014E00023F06047BD0C15EA230538BF3D4634465E
:1014F0004FEAD37EC3F3807C6368BEEBD37F23F0D7
:101500006042DDD1974203D1C3F380739C450AD179
:10151000974205E01C46EFE7AA4206D013469D42DB
:101520002CBF00230123002BCFD12368A046002B22
:10153000F0D12160BDE8F081743F0008683D0008EB
:101540002C4000084D40000808B5034A034B40F208
:101550005E31034802F06AFA443D0008EC3F00089F
:101560002C40000808B503680B60C388016033B9DC
:10157000044B054A4FF4C761044802F057FA013B97
:10158000C38008BDBC3F0008B83D00082C400008DF
:1015900070B50C4600F10C05616831B9E38A002092
:1015A00061F30903E382002170BD0E682846FFF74E
:1015B000D9FF6660F0E7000008B5426832B10B4B16
:1015C0000B4A40F22F410B4802F030FAC37DC3F3BF
:1015D0008401013161F38603C375C38A62F3090391
:1015E000C3821B0A62F3C713C37508BD0840000815
:1015F000743D00082C4000082DE9F047089E32B9E0
:101600001F4B204A40F239511F4802F00FFA4FF4A5
:101610007F4901F007054FEAD6082A4406F007067D
:1016200000EBD100954201D1BDE8F08705F0070E2F
:1016300006F0070AD645774638BF5746511BC7F113
:1016400008078F4228BF0F46EC08045D08EBD6015F
:1016500013F801C004FA0EF429FA07FE24FA0AF47A
:101660005FFA8EFE8CEA04044EFA0AFE04EA0E04C7
:101670008CEA040C03F801C03D443E44D2E700BFAD
:10168000883F00088C3D00082C4000082DE9F041FF
:1016900006460F4600254FF6FF7441F221082A4600
:1016A00030463946FEF75CFD0823C0B284EA0024C8
:1016B00014F4004F4FEA4404A4B203F1FF3318BFFF
:1016C00084EA080413F0FF03F2D10835402DE6D177
:1016D0002046BDE8F081000010B541F221040A4423
:1016E000914200D110BD11F8013B80EA032008238C
:1016F00010F4004F4FEA400080B203F1FF3318BFEF
:10170000604013F0FF03F3D1EAE700002DE9F04F4A
:1017100085B08A468DE80C00BDF83C40814630B962
:1017200040F26E31484B494A494802F07FF911F0C6
:10173000604F04D0474B454A40F26F31F4E7009BBD
:10174000002B7ED024B10E9B002B7AD0072C28D8FA
:1017500009F10C00FFF772FE054628B96FF002058B
:10176000284605B0BDE8F08F14220021FFF710FED7
:1017700022460E9905F10800FFF7F8FD631C2B7453
:10178000009B2C441B78294603F01F0363F03F03A2
:1017900023724AF000436B604846FFF77BFE012549
:1017A000DEE74FF000084FF0800B46464546019BB0
:1017B0001B0A029300F10C0303930398FFF73EFE0C
:1017C00007460028CAD014220021FFF7E1FDB6BB6E
:1017D00002229DF804303B729DF808307B720E9B0C
:1017E000711E1944B4420AD9B818013211F801EF38
:1017F000D2B20136072A80F808E0B6B2F2D1B4427C
:1018000008BF4FF0400B009BB8181978013201F067
:101810001F0141EA48114BEA010303724AF00043F9
:101820007B603A7439464846FFF734FE0135B442CE
:101830002DB288F001084FF0000BBED190E70022D6
:10184000CDE76FF001058BE7743F0008583D0008B5
:101850002C400008983F00082DE9F0471E46CB8A2F
:101860009146C3F30902062A80460F4619D0134653
:101870000021B0B28DB25A1992B2052A09D9A842F4
:1018800010D8FA8A034463F30902FA820120BDE802
:10189000F087A842F3D919F801403A44947601310F
:1018A000E8E70025FB8A7C68C3F309001C23821F3C
:1018B000B2FBF3FA03FB1A2A1FFA8AF27CB3012166
:1018C0002368002B39D1B31F03441C20B3FBF0F372
:1018D00001339BB299420CD2BAF1000F09D14046B4
:1018E000FFF7ACFD08B1C0F800A0206008B30446C3
:1018F00000224FF0000AB6B2B54230D21346691E3C
:101900004944E018013311F801EF9BB201351C2B5B
:1019100080F804E0ADB214D0AE42F2D8ECE7404615
:10192000FFF78CFD044608B1002303607C60002CA7
:10193000DED16FF00200BDE8F087013189B21C46AC
:10194000BEE7AE42D8D94046FFF778FD08B1C0F8EF
:1019500000A020600028ECD004460022CCE7FB8ADF
:10196000C3F30902164466F30903FB828EE7000005
:10197000F8B50E4615461F46044628B9144B154ABD
:101980004F21154802F052F824220021FFF700FDF4
:10199000069B6A096360079B002023624FF6FF7372
:1019A0009A4228BF1A46A7602070A061E06197B2F2
:1019B00004F10C05824205D100232B60278263824B
:1019C000A382F8BD2E60013035462036F2E700BF15
:1019D000703F0008E43C00082C40000808B528B916
:1019E0007321084B084A094802F020F8037823B90C
:1019F0004BB2002B01DD017008BD054B024A7D2171
:101A0000F1E700BF743F0008F03C00082C400008DC
:101A1000B83E0008007870472DE9F7430D9E074651
:101A200019461046BDF828900B9D9DF83040BDF832
:101A3000388016B9B8F1000F43D11F2C41D83B783C
:101A4000D3B9B8F1070F39D839F0030339D1424679
:101A500031464FF6FF70FFF73FFE4FEA092920F0AD
:101A6000010009F44079400449EA0464400C44EA66
:101A700040244FF6FF730DE043EA0923B8F1070F46
:101A800043EA0464F5D9FFF701FE42463146FFF709
:101A900023FE03468DE840012A4621463846FFF7DB
:101AA00035FE0DB9FFF750FD2B780133DBB21F2B4C
:101AB00088BF00232B7003B0BDE8F0836FF00300F4
:101AC000F9E76FF00100F6E72DE9F7430E9F814635
:101AD0000B9D9DF830009DF83480BDF83C6007B93F
:101AE000C6BB1F2836D899F800E0BEF1000F34D0ED
:101AF0000C0244F080049DF8281044EAC83444EAFB
:101B0000014444EA0E04072E44EA006415D919463C
:101B10001046FFF7BBFD32463946FFF7DDFD0346B1
:101B2000019600972A4621464846FFF7EFFDB8F197
:101B3000010F0CD125B9FFF707FD4FF6FF73EFE753
:101B40002B780133DBB21F2B88BF00232B7003B02F
:101B5000BDE8F0836FF00100F9E76FF00300F6E7EE
:101B6000C06900B104307047C1690C300B68036173
:101B7000FFF7F8BC2DE9F84FD0F818A00546164637
:101B80001F4654464FF00009DFF8608000F10C0B4F
:101B90000CB9BDE8F88FD4E90223B21A67EB03034E
:101BA000994508BF90451FD2AB6921469C42284603
:101BB0000DD1FFF7EDFCAB6921461B685846AB61C0
:101BC000FFF7D0FCAC692346A2461C46E0E7FFF7CE
:101BD000DFFC23682146CAF800305846FFF7C2FCF4
:101BE0005446DAF80030EFE72368EDE780841E0002
:101BF0002DE9F04F8BB00D4614460793DDF8509059
:101C00008246002800F06481B9F1000F00F0608185
:101C1000531E3F2B00F25C81012A03D1079B002B4E
:101C200040F056810023BAF814600893F600B542DC
:101C3000099380F053812B199E420AD2761B16F02D
:101C4000FF0607D140F26751AA4BAB4AAB4801F0FF
:101C5000EDFE2646DAF80C3023B9DAF81030002B06
:101C600000F0A5802F2D31D8C5F1300846454FF042
:101C7000000334BFB0465FFA88F80093294608ABEA
:101C80004246DAF80800FFF7B7FCA6EB0807454420
:101C9000FFB24FF0300BBAF8143003F10053063B9B
:101CA000DB000293DAF80C300593059B002B51D032
:101CB00087B9DAF81000002861D0002F5FD0AB455B
:101CC00050D98F4B8C4A40F2A651BFE737464FF0B0
:101CD0000008DEE7029B23B98A4B874A4FF4B161C3
:101CE000B4E7029BE02B28BFE02306935B44AB42A2
:101CF00004931DD95B1B9F4226BFDBB2039303975E
:101D0000AB4504D97E4B7C4A40F291519EE7059841
:101D1000CDF8008008ABA5EB0B01039A0430FFF768
:101D20006BFC039B9844FF1A1D445FFA88F8FFB2CE
:101D3000049B9B4504D3744B6F4A40F29B5185E74B
:101D4000029B069ADDF810B09B1A0293059B1B6854
:101D50000593AAE7029BBB42ABD26C4B664A40F2AA
:101D6000A15173E7CDF800803A46A5EB0B0108AB13
:101D7000B8443D44FFF740FC00275FFA88F8BAF802
:101D80001430B5EBC30F04D9614B5B4A40F2B1513B
:101D90005CE7B8F1400F04D95E4B574A40F2B251AC
:101DA00054E767B15C4B544A40F2B3514EE700939D
:101DB000324608AB2946DAF80800FFF71DFC731E0F
:101DC0003F2B35B201D8A64204DD544B544A40F2B1
:101DD00035213BE760070AD00AAB03EBD40111F8C9
:101DE000083C624202F00702134101F8083C082C4B
:101DF00021D9102C21D9202C8CBF08230423079A29
:101E0000002A6DD0B4EBC30F6CD0082C04F1FF3264
:101E100015D89DF8203023FA02F2D10706D54FF0ED
:101E2000FF3202FA04F423438DF820309DF820306D
:101E300089F800304EE00123E1E70223DFE7102CB0
:101E400011D8BDF8203023FA02F2D20706D54FF0A0
:101E5000FF3202FA04F42343ADF82030BDF82030FD
:101E6000A9F8003036E0202C0ED8089921FA02F2A9
:101E7000D30705D54FF0FF3303FA04F40C4308945D
:101E8000089BC9F8003025E0402C1CD0DDE908672C
:101E900030463946FEF764F9002100F0010050EAAF
:101EA00001030BD0224601200021FEF765F94042D4
:101EB00061EB410106430F43CDE90867DDE90823E3
:101EC000C9E9002306E0174B154A4FF42071BDE61F
:101ED0006FF0010528460BB0BDE8F08F1D46F9E70D
:101EE000012CA3D0082CA1D9102CB7D9202CE5D8CF
:101EF000C6E700BFC43D00089C3D00082C40000818
:101F0000E63D0008D33D00080B3E0008333E0008C4
:101F10005A3E0008883E0008A03E0008BA3E00086D
:101F20001C3D0008B83E000830B585B030B940F21D
:101F3000B121234B234A244801F078FD23B9234BD8
:101F4000204A40F2B221F6E7402A04D9204B1D4A2C
:101F500040F2B621EFE722B91D4B1A4A4FF42F7118
:101F6000E9E70024012A0294039417D11B788DF825
:101F7000083053070AD004AB03EBD20313F8084C24
:101F8000554205F00705AC4003F8084C00910346A4
:101F9000002102A8FFF730FB05B030BD082AE5D9C3
:101FA000102A03D81B88ADF80830E2E7202A02D8AF
:101FB0001B680293DDE7D3E90045CDE90245D8E788
:101FC000F43E0008303D00082C4000080F3F000898
:101FD000B83E000870B50C4600F10C05E16819B96F
:101FE000A1602161A18270BD0E682846FFF7BAFA90
:101FF000E660F3E72DE9F04FD1F8009091B0C9F316
:10200000C01604460D46CDE90223002E50D0C9F378
:10201000C03BC9F30626B9F1000F80F29F8119F089
:10202000C04F40F09B812B7B002B00F09781BBF1D0
:10203000020F03D02278B24240F0938109F07F0270
:10204000BBF1020F059236D119F07F0FC9F30F2AA9
:1020500001D10AF0030A2B447606059A93F803800F
:1020600046EA0B4646EA82465FEAD81346EA0A0683
:10207000069300F09A800022002310A961E908234A
:10208000059B6768009352465B462046B847002888
:1020900000F08880A7698FB9314604F10C00FFF782
:1020A000DBF90746D0B96FF0020011B0BDE8F08F40
:1020B0004FF0020BAFE7C9F3074ACCE73B699E42FA
:1020C0000DD03F68002FF9D1314604F10C00FFF725
:1020D000C3F907460028E6D0A3693B60A761DDE9A4
:1020E0000801FFF7D3FAB882F97D08F01F06C1F3A3
:1020F0008401711A89B20FFA81FEBEF1000FB8BFD8
:1021000001F1200EC9F30461D7E90223B8BF0FFA29
:102110008EFE079152EA030100F02F81DDE90201F2
:10212000801A61EB03010B46002102469E4899424A
:1021300008BF9042C0F02181069B002B3FD0BEF12A
:10214000010F00F31A8118F0400F38D0DDE90223A7
:10215000C7E90223202200210DEB0200FFF718F946
:10216000DDE90223CDE908232B1D0A932B7B2046B2
:10217000013BDBB2ADF834309DF81C30ADF836A031
:102180008DF83A309DF814308DF838B08DF83B302A
:102190008DF83960A36808A998473846FFF70CFA0C
:1021A000002082E76FF00B007FE7A76917B96FF097
:1021B0000C007AE73B699E4296D03F68F6E7FB7DCC
:1021C000C8F34012B2EBD31F40F0CE80C3F38403B8
:1021D000B34240F0CC8006992B7B4FEA981279B33A
:1021E000D2073CD4032B40F2C580DDE90223C7E9C6
:1021F00002232B7BAE1D033BDBB23246394604F192
:102200000C00FFF729FB002808DA39462046FFF7C3
:10221000BFF93846FFF7D0F9032046E7AB883B8388
:102220002A7B033AD2B2B88A3146FFF755FAFB7DD2
:10223000B882DA43C2F3C01262F3C713FB75AFE78B
:102240006AB92E1D013BDBB23246394604F10C005F
:10225000FFF702FB0028D8DB2A7B013AE2E7FA8A83
:10226000013BC2F30902052AD9B250D80023281D28
:1022700099420AD907EB020E10F801CB0132013363
:10228000062A8EF81AC0DBB2F2D18B4228BF002397
:10229000DDE9028907F11A02CDE908890A927A6814
:1022A0003CBF04335B190B920C93FB8AADF836A04C
:1022B000C3F3090319449DF81C30ADF834108DF8B0
:1022C0003A309DF814308DF838B08DF83B3000234B
:1022D0008DF839607B602A7BB88A013A291DFFF7A7
:1022E000FBF93B8BB882834203D1A36808A920463F
:1022F000984708A92046FFF76DFE3846FFF75CF9BE
:10230000B88A3B8B984214BF11200020CDE6786834
:1023100010B34FF0060E03689BB9A2EB0E021B2A06
:1023200013D80332024405F1040E1F309942ACD990
:102330001EF801CB013302F801CF9042DBB2F5D198
:10234000A3E70EF11C0E1846E5E7184B184A40F2B9
:10235000B311184801F06AFB034696E76FF00900D5
:10236000A3E66FF00A00A0E66FF00D009DE66FF0A7
:102370000E009AE66FF00F0097E6FB7D394668F392
:1023800086036FF3C713FB752046FFF701F9069B21
:10239000002B7FF4D8AEFB7DC3F38402013262F3DD
:1023A0008603FB7503E700BF80841E00243F0008FE
:1023B000083D00082C4000082DE9F0414E4EB04287
:1023C00040F086804D4CDFF838E1E56945F0007556
:1023D000E561E469846AD4F8007207EA0E0747F001
:1023E0000107C4F80072D4F8005205EA0E0545F062
:1023F000010545EA0121C4F80012002A6AD0002133
:102400000F46C4F81C12C4F80412C4F80C12C4F825
:10241000141204EBC10501311C29C5F84072C5F83E
:102420004472F6D14FF0000E4FF0010C964510D1DA
:10243000826AB042D2F8003223F00103C2F80032BF
:1024400058D12E4BDA6922F00072DA61DB69BDE8FF
:10245000F0819F781D8817F0010F18BFD4F804820F
:102460000CFA05F11CBF41EA0808C4F8048217F011
:10247000020F18BFD4F80C8204EBC5051CBF41EA5B
:102480000808C4F80C827F0748BFD4F8147203F11F
:102490000C0344BF0F43C4F8147253F8087C0EF1C8
:1024A000010EC5F8407253F8047CC5F84472D4F8A4
:1024B0001C522943C4F81C12B8E70021846AC4F8EE
:1024C0001C12C4F80412C4F80C12C4F81412A9E7C0
:1024D000002AF2D10022836AC3F84022C3F84422C2
:1024E000C3F80422C3F814220122C3F80C22C3F853
:1024F0001C229DE7BDE8F081B819002000100240C1
:102500000000FFFF184A08B5916A8B688B6013F0D2
:10251000010105D013F00C0F14BF4FF480310121DD
:10252000D80506D513F4406F14BF41F4003141F0D3
:102530000201D80306D513F4402F14BF41F48021C3
:1025400041F00401D3690BB107489847202383F376
:1025500011880021054800F087FB002383F31188D0
:10256000BDE8084000F066BDB8190020C019002081
:1025700038B5124CA36ADD68AA0712D05A6922F056
:1025800002025A61A36913B1012120469847202312
:1025900083F3118800210A4800F066FB002383F3CF
:1025A0001188EB0606D51021A36AD960236A0BB106
:1025B00002489847BDE8384000F03CBDB8190020FB
:1025C000C819002038B5124CA36A1D69AA0712D099
:1025D0005A6922F010025A61A36913B10221204600
:1025E0009847202383F3118800210A4800F03CFB20
:1025F000002383F31188EB0606D51021A36A196125
:10260000236A0BB102489847BDE8384000F012BD7C
:10261000B8190020C819002038B50F4CA36A5D68AE
:102620002A075D600AD5032222701A6822F002028E
:102630001A60636A13B10021204698476B0706D5DC
:10264000A36A9969236A13B1090403489847BDE84E
:10265000384000F0EFBC00BFB819002010B50F4C97
:10266000204600F06FF90E4B0B211320A36200F0FF
:1026700049F90B21142000F045F90B21152000F039
:1026800041F90B21162000F03DF900232046BDE85A
:1026900010401A460E21FFF78FBE00BFB819002068
:1026A000006400400F4B10B59842044605D10E4B14
:1026B000DA6942F00072DA61DB690122A36A1A600A
:1026C000A36A5A68D20707D5626851681268D9614F
:1026D0001A60064A5A6110BD0121082000F0F8F97D
:1026E000EEE700BFB8190020001002405B87010030
:1026F00003291AD8DFE801F0020A0F14836A9B68E5
:1027000013F0E05F14BF012000207047836A9868CF
:10271000C0F380607047836A9868C0F3C0607047F8
:10272000836A9868C0F3007070470020704700000B
:1027300010B503291FD8DFE801F0021F2327816AA3
:102740008B68C3F30163183301EB03131078810620
:102750001ED55468C0F30011490041EAC40141F09C
:10276000040100F00F005860906841F0010198608A
:10277000D268DA60196010BD836A03F5C073E5E7BB
:10278000836A03F5C873E1E7836A03F5D073DDE775
:102790009488C0F30011490041EA4451E1E7000088
:1027A00001290CD003D3022910D000207047836A7E
:1027B000DA68920701D1186903E001207047836A43
:1027C000D86810F0030018BF01207047836AF2E751
:1027D00010B539B9836AD96889071BD11B699B0772
:1027E00004D110BD012915D0022948D1816AD1F840
:1027F000C031D1F8C401D1F8C8411461D1F8CC413D
:10280000546120240C610C69A40717D14C6944F071
:10281000100412E0816AD1F8B031D1F8B401D1F8D6
:10282000B8411461D1F8BC4154612024CC60CC681B
:10283000A40703D14C6944F002044C6111795C088F
:1028400064F304119C0864F34511117189064BBFB0
:1028500091681189DB085B0D4CBF63F31C0163F3C6
:102860000A01137948BF916060F3030313714FEAC3
:1028700010234FEA104058BF11811370508010BDD3
:1028800000231A4610B51C495A50CC180833802B27
:102890006260F9D1194B9A6942F07D029A619B6995
:1028A0000268174BDA6082685A6042681A60C26830
:1028B00003F58063DA6042695A6002691A608269CE
:1028C000C3F80C24026AC3F80424C269C3F80024C4
:1028D000426AC3F80C28C26AC3F80428826AC3F8A3
:1028E0000028026BC3F80C2C826BC3F8042C426BDB
:1028F000C3F8002C10BD00BFE419002000100240F6
:102900000008014000F16043090103F56143C9B2C9
:1029100083F80013012300F01F024009800000F13A
:102920006040934000F56140C0F88031036070471B
:10293000090100F16040C9B200F56D4001767047B1
:10294000FFF78CBE01230370002300F108028260B0
:10295000C26000F110024360026142618361C361A1
:10296000036243627047000010B52023044683F3DE
:102970001188022341600370FFF794FE0323237044
:10298000002383F3118810BD2DE9F0411F46044652
:102990000D461646202383F3118800F1080823789A
:1029A000042B0ED029462046FFF7A2FE48B1204650
:1029B00032462946FFF7BCFE002080F31188BDE8AF
:1029C000F0813946404600F033F90028E7D0002373
:1029D00083F31188BDE8F0812DE9F0411F460446DC
:1029E0000D461646202383F3118800F11008237842
:1029F000042B0ED029462046FFF7D2FE48B12046D0
:102A000032462946FFF7E4FE002080F31188BDE836
:102A1000F0813946404600F00BF90028E7D000234A
:102A200083F31188BDE8F0810022024B1B605B60DC
:102A30009A607047641A0020002382680374054B73
:102A40001B6899689142FBD25A680360426010602B
:102A500058607047641A002008B5202383F311885A
:102A6000037C032B05D0042B0DD02BB983F31188E5
:102A700008BD002243691A604FF0FF334361FFF73E
:102A8000DBFF0023F2E790E80C001A600268536055
:102A9000F2E70000002382680374054B1B68996805
:102AA0009142FBD85A6803604260106058607047DA
:102AB000641A0020054B196908741868026853608D
:102AC0001A60186101230374FDF75ABD641A0020CF
:102AD00030B54B1C87B005460A4C10D023690A4A12
:102AE00001A800F0DDF82846FFF7E4FF049B13B1CE
:102AF00001A800F0EFF82369586907B030BDFFF76F
:102B0000D9FFF8E7641A0020592A000838B50C4D9F
:102B100041612B6981689A680446914203D8BDE8F7
:102B20003840FFF789BF1846FFF786FF01232C6165
:102B3000014623742046BDE83840FDF721BD00BFA3
:102B4000641A0020044B1A681B6990689B689842BD
:102B500094BF002001207047641A002010B5084C73
:102B6000236820691A6854602260012223611A7464
:102B7000FFF790FF01462069BDE81040FDF700BD5A
:102B8000641A002008B5FFF7DDFF18B1BDE8084062
:102B9000FFF7E4BF08BD0000826002220274002239
:102BA000427470478368A3F13C0243F80C2C02691D
:102BB00043F83C2C426943F8382C074A43F81C2C54
:102BC000C268A3F1180043F8102C022203F8082C65
:102BD000002203F8072C70479105000810B5202348
:102BE00083F31188FFF7DEFF00210446FFF78EFF15
:102BF000002383F31188204610BD0000024B1B699F
:102C000058610F20FFF756BF641A0020202383F37A
:102C10001188FFF7F3BF000008B50146202383F3B6
:102C200011880820FFF754FF002383F3118808BDA3
:102C300049B1064B42681B6918605A6013604360D3
:102C40000420FFF745BF4FF0FF307047641A0020A3
:102C50000368984206D01A680260506059611846AD
:102C6000FFF7EABE7047000038B504460D462068FD
:102C7000844200D138BD036823605C604561FFF782
:102C8000DBFEF4E7054B03F114025A619A614FF041
:102C9000FF32DA6100221A62704700BF641A002016
:102CA00010B5C2600A4A036153699C68A1420CD8FE
:102CB0005C68036044602060586081609868411AD5
:102CC00099604FF0FF33D36110BD091B1B68ECE71F
:102CD000641A0020036881689A680A449A6042680E
:102CE000136003685A6000234FF0FF32C360014B4A
:102CF000DA617047641A002000207047FEE7000088
:102D0000704700004FF0FF3070470000BFF34F8F57
:102D1000024AD368DB07FCD4704700BF00200240A2
:102D200008B5074B1B7853B9FFF7F0FF054B1A693D
:102D3000120641BF044A5A6002F188325A6008BD47
:102D4000B41A0020002002402301674508B5054B56
:102D50001B7833B9FFF7DAFF034A136943F08003A6
:102D6000136108BDB41A0020002002407F289ABFDA
:102D700000F58030C0020020704700004FF4006072
:102D800070470000802070477F2808B50BD8FFF7F8
:102D9000EDFF00F500630268013204D10430834284
:102DA000F9D1012008BD002008BD00007F2810B522
:102DB00004461CD8FFF7AAFFFFF7B2FFF3220D4B22
:102DC000DA6002221A61FFF7D1FF58611A6942F0F6
:102DD00040021A61FFF79AFF4FF4006100F0E4F837
:102DE000FFF7B4FF2046BDE81040FFF7CDBF00203D
:102DF00010BD00BF002002402DE9F84312F001038E
:102E0000144606D040F241221F4B1A600020BDE854
:102E1000F88385181D4A954204D940F246211A4A82
:102E20001160F3E7FFF77CFFFFF770FF4FF0010938
:102E3000DFF86880451A012C05EB01060F4604D81F
:102E4000FFF784FF0120BDE8F883C8F8109031F83F
:102E5000023B3380FFF75AFF0020C8F81000338888
:102E60003A889BB29A420DD040F25D22064B1A601E
:102E7000074B1E60074B1C60074B1F60FFF766FF88
:102E8000BDE8F883023CD6E7B01A0020FFFF030834
:102E9000A41A0020AC1A0020A81A0020002002402A
:102EA000084908B50B7828B153B9FFF739FF01235A
:102EB0000B7008BD23B1BDE808400870FFF746BF9E
:102EC00008BD00BFB41A002038B500F059F94FF41E
:102ED0007A730C490C4A0C6A116803FB04F38B42A9
:102EE0000A49D1E9004504D2003445F10105C1E9A0
:102EF0000045E41845F10005136000F04BF9204649
:102F0000294638BD641A0020B81A0020C01A0020D3
:102F100008B5FFF7D9FF4FF47A720023FDF738F9AF
:102F200008BD00BF10B5094C0439013AD2B2FF2ADE
:102F300000D110BD53089800043054F823300059D4
:102F40009BB243EA004341F8043FEEE7046C0040C3
:102F500030B50748013AD2B2FF2A00D130BD0D8802
:102F6000540840F82450A3004C8804331C50F1E767
:102F7000046C004007B5012201A90020FFF7D2FF31
:102F8000019803B05DF804FB13B50446FFF7F2FFA8
:102F9000A04206D002A941F8044D01220020FFF70B
:102FA000D7FF02B010BD00007047000045F2555237
:102FB000064B1A6002225A6040F6FF729A604CF685
:102FC000CC421A600122024B1A7070470030004058
:102FD000C91A0020034B1B781BB14AF6AA22024BE8
:102FE0001A607047C91A002000300040034B1B686C
:102FF0009B0042BF0122024B1A707047241002400E
:10300000C81A00204FF08072014B1A60704700BF51
:1030100024100240014B1878704700BFC81A0020E6
:10302000EFF30983203383F30988002383F31188A6
:103030007047000010B5202383F311880D4B5B68A7
:1030400013F4006312D0EFF309844FF0807344F857
:10305000043CA4F1200383F30988FFF773FD18B142
:10306000054B44F8083C10BD044BFAE783F3118884
:1030700010BD00BF00ED00E0A1050008A405000898
:1030800070470000FEE70000084A094B09498B42DF
:1030900004D30021084A934205D3704752F8040F25
:1030A00043F8040BF3E743F8041BF4E7AC410008D2
:1030B000542400205424002054240020FEE7000063
:1030C00010B5174CFFF7B0FCFFF7DCFD8022154967
:1030D0002046FFF761FD012344F8180C0374124BDE
:1030E000124AD96821F4E0610904090C0A43104925
:1030F000DA60CA6842F08072CA600E490A6842F01B
:1031000001020A601022DA77202283F822200023AD
:1031100083F3118862B6BDE810400748FFF75EBD33
:103120008C1A00206840000800ED00E00003FA055A
:10313000F0ED00E0001000E070400008F8B50F4C22
:10314000226A01322262224652F8141F9142154629
:1031500006D020268B68013B8B6063699A6802B1B8
:10316000F8BD1968DF68DA604D60616182F311882B
:103170001869B84786F31188EFE700BF641A00208A
:10318000EFF3118020B9EFF30583202282F3118839
:103190007047000010B558B9EFF30584C4F3080474
:1031A00014B180F3118810BDFFF7ECFC84F3118893
:1031B00010BD000000F030B808B500F069F9FFF765
:1031C0007FFFBDE80840FFF711BF00007047000017
:1031D0004FF0FF310E4B1A6919611A6900221A610A
:1031E0001869D868D960D968DA60DA68DA6942F0B3
:1031F0008052DA61DA69DA6942F00062DA61054A1E
:10320000DB69136843F48073136000F021B900BFD9
:1032100000100240007000401C4B1A6842F001028E
:103220001A601A689007FCD55A6822F003025A60A7
:103230005A6812F00C02FBD1196801F0F90119600B
:103240005A601A6842F480321A601A689103FCD5F9
:103250004EF63162DA625A6842F4E8125A601A682D
:1032600042F080721A601A689201FCD51221084A55
:103270005A60084A11605A6842F002025A605A685D
:1032800002F00C02082AFAD1704700BF0010024079
:1032900000641D0000200240084A08B55369116807
:1032A0000B4003F00103536123B1054A13680BB1CE
:1032B00050689847BDE80840FFF7BCBE00040140D5
:1032C000E4190020084A08B5536911680B4003F05F
:1032D0000203536123B1054A93680BB1D068984744
:1032E000BDE80840FFF7A6BE00040140E419002035
:1032F000084A08B5536911680B4003F00403536191
:1033000023B1054A13690BB150699847BDE80840DD
:10331000FFF790BE00040140E4190020084A08B5F8
:10332000536911680B4003F00803536123B1054A48
:1033300093690BB1D0699847BDE80840FFF77ABEA2
:1033400000040140E4190020084A08B553691168D7
:103350000B4003F01003536123B1054A136A0BB10C
:10336000506A9847BDE80840FFF764BE000401407A
:10337000E4190020174B10B55C691A68144004F476
:1033800078725A61A30604D5134A936A0BB1D06AC6
:103390009847600604D5104A136B0BB1506B9847E1
:1033A000210604D50C4A936B0BB1D06B9847E2050C
:1033B00004D5094A136C0BB1506C9847A30504D58A
:1033C000054A936C0BB1D06C9847BDE81040FFF7ED
:1033D00031BE00BF00040140E41900201A4B10B5B3
:1033E0005C691A68144004F47C425A61620504D591
:1033F000164A136D0BB1506D9847230504D5134A37
:10340000936D0BB1D06D9847E00404D50F4A136E4D
:103410000BB1506E9847A10404D50C4A936E0BB1C2
:10342000D06E9847620404D5084A136F0BB1506FF1
:103430009847230404D5054A936F0BB1D06F984782
:10344000BDE81040FFF7F6BD00040140E41900207C
:10345000062108B50846FFF755FA06210720FFF7B1
:1034600051FA06210820FFF74DFA06210920FFF73F
:1034700049FA06210A20FFF745FA06211720FFF72F
:1034800041FABDE8084006212820FFF73BBA0000BA
:1034900008B5FFF79DFE0648FFF7F2F9FFF750FA6F
:1034A00000F03AF8FFF792FEBDE8084000F070B86F
:1034B00090400008026843681143016003B1184757
:1034C00070470000143000F0FFB900004FF0FF33E8
:1034D000143000F0F9B90000383000F075BA00007F
:1034E0004FF0FF33383000F06FBA0000143000F0B6
:1034F000C5B900004FF0FF31143000F0BFB9000033
:10350000383000F01FBA00004FF0FF32383000F0C2
:1035100019BA00000020704700F00AB90F4B37B508
:103520000360002343608360C360012304461546A3
:1035300003744FF4007200900B4600F15C011430EC
:1035400000F072F900942B464FF4007204F51771E5
:1035500004F1380000F0EAF903B030BDCC400008B7
:1035600038B5C36904460D461BB904210844FFF76A
:10357000A1FF294604F1140000F064F9002806DADE
:10358000201D4FF48061BDE83840FFF793BF38BD80
:1035900000F00EB808B5202383F31188FFF7CEFDA5
:1035A000002383F31188BDE80840FFF743BD000006
:1035B000054B064A08215A6000229A6007220B2018
:1035C0001A60FFF7B5B900BF10E000E03F19010035
:1035D000026843681143016003B118477047000057
:1035E000024AD36843F0C003D360704700440040F0
:1035F000024AD36843F0C003D360704700480040DC
:103600002DE9F041D0F85C640546F7683368DA05C7
:103610009CB20DD5202383F311884FF40071043040
:10362000FFF7D6FF6FF480733360002383F31188B4
:10363000202383F3118805F1040814F02F0333D1FC
:1036400083F31188380615D5210613D5202383F37B
:10365000118805F1380000F09DF9002846DA0821AC
:10366000281DFFF7B5FF4FF67F733B40F360002343
:1036700083F311887A060ED563060CD5202383F3D5
:103680001188EA6C2B6D9A4202D12B6C002B2FD142
:10369000002383F31188D5F86424D368002B31D03C
:1036A000BDE8F04110691847230713D014F0080F44
:1036B0000CBF00218021E00748BF41F02001A20794
:1036C00048BF41F04001630748BF41F48071404664
:1036D000FFF77EFFA406736805D595F860142846A9
:1036E0001940FFF73DFF3468A4B2A6E77060BEE75B
:1036F00027F040073F041021281D3F0CFFF768FF0B
:10370000F760C5E7BDE8F08108B50348FFF778FF2B
:10371000BDE80840FFF78EBC801B002008B50348B9
:10372000FFF76EFFBDE80840FFF784BCE81F0020EC
:1037300010B5094C094A20460021FFF7EFFE084B5F
:10374000084AC4F85C34084C00212046FFF7E6FE26
:10375000064BC4F85C3410BD801B0020E135000826
:1037600000440040F1350008E81F002000480040F8
:10377000F8B5154682680B46AA428169066938BFCA
:103780008568761AB542044607D218462A46FDF7E0
:10379000EDFDA3692B44A3610DE011D93246184613
:1037A000FDF7E4FDAF1B3A46E1683044FDF7DEFD6E
:1037B000E2683A44A261A36828465B1BA360F8BD97
:1037C00018462A46FDF7D2FDE368E4E72DE9F0410B
:1037D0000446154683682669934238BF8568406968
:1037E0000F46361AB54206D22A46FDF7BFFD636979
:1037F0002B4463610DE012D93246A5EB0608FDF7B4
:10380000B5FD4246B919E068FDF7B0FDE2684244F3
:103810006261A36828465B1BA360BDE8F0812A466D
:10382000FDF7A4FDE368E4E710B50024C361029B43
:103830000A44006040608460C1608161416102614E
:10384000036210BD08B582694369934201D1826861
:1038500082B98268013282605A1C426119704269E1
:1038600003699A4201D3C36843610021FFF7F0F96D
:10387000002008BD4FF0FF3008BD000070B52023C8
:1038800004460E4683F31188A568A5B1A368A26912
:10389000013BA360531CA36115782269934224BFA6
:1038A000E368A361E3690BB120469847002383F3E3
:1038B0001188284670BD31462046FFF7B9F9002827
:1038C000E2DA85F3118870BD2DE9F74F05460F4602
:1038D00090469A46D0F81C90202686F311884FF027
:1038E000000B144664B1224639462846FFF740FFD4
:1038F000034668B951462846FFF79AF90028F1D0E7
:10390000002383F31188A8EB040003B0BDE8F08F17
:10391000B9F1000F03D001902846C847019B8BF3F3
:103920001188E41A1F4486F31188DBE7C361009B0A
:10393000C160816141611144006040608260016149
:1039400003627047F8B504460E461746202383F3FA
:103950001188A568A5B1A368013BA36063695A1CDF
:1039600062611E70236962699A4224BFE3686361E1
:10397000E3690BB120469847002080F31188F8BD19
:1039800039462046FFF754F90028E2DA85F311881A
:10399000F8BD00008369426910B59A4201D182687E
:1039A0007AB98268013282605A1C82611C7803698C
:1039B0009A4201D3C36883610021FFF749F9204689
:1039C00010BD4FF0FF3010BD2DE9F74F05460F46F3
:1039D00090469A46D0F81C90202686F311884FF026
:1039E000000B144664B1224639462846FFF7EEFE26
:1039F000034668B951462846FFF71AF90028F1D066
:103A0000002383F31188A8EB040003B0BDE8F08F16
:103A1000B9F1000F03D001902846C847019B8BF3F2
:103A20001188E41A1F4486F31188DBE71FB51C4692
:103A3000094B05461B68D86852B1084B8DE80A004F
:103A400002922B4622460649FDF7AEFC00F042F8F2
:103A5000044B1A46F2E700BF14080020F4400008A7
:103A600001410008E73B000810B5013902449042CB
:103A700001D1002010BD10F8013B11F8014FA34205
:103A8000F5D0181B10BD00002DE9F8430746884605
:103A900091461E468BB10D46A8EB0500B54207EBDB
:103AA000000402D20020BDE8F88332464946204691
:103AB000FFF7DAFF18B1013DEEE7BDE8F8832046D5
:103AC000BDE8F883034611F8012B03F8012B002A07
:103AD000F9D1704708B5062000F02CF80120FFF757
:103AE0000DF900001F2938B504460D4604D91623E8
:103AF00003604FF0FF3038BD426C12B152F82130F4
:103B00004BB9204600F030F82A4601462046BDE871
:103B1000384000F017B8012B0AD0591C03D11623E6
:103B20000360012038BD0024284642F8254098470C
:103B3000002038BD024B01461868FFF7D3BF00BF15
:103B40001408002038B50023064C054608461146E7
:103B50002360FFF7D7F8431C02D1236803B12B6021
:103B600038BD00BF50240020FFF7C6B840A2E4F1E2
:103B7000646891064E6F20617070207369670A0057
:103B8000426164206677206C656E677468202575D5
:103B90000A0042616420626F6172645F696420257B
:103BA000752073686F756C642062652025750A0046
:103BB0004261642061707020435243203078253088
:103BC00038783A3078253038782030782530387891
:103BD0003A3078253038780A00476F6F642066697C
:103BE000726D776172650A007265636569766564F6
:103BF0005F756E697175655F69645F6C656E203CA9
:103C00002055415643414E5F50524F544F434F4C05
:103C10005F44594E414D49435F4E4F44455F4944CF
:103C20005F414C4C4F434154494F4E5F554E4951B3
:103C300055455F49445F4D41585F4C454E47544898
:103C4000002E2E2F2E2E2F546F6F6C732F41505F2E
:103C5000426F6F746C6F616465722F63616E2E6367
:103C6000707000616C6C6F63617465645F6E6F642B
:103C7000655F6964203C3D20313237006F72672EEA
:103C80006172647570696C6F742E61705F706572BB
:103C90006970685F5A75626178474E53530000003F
:103CA000766F69642068616E646C655F616C6C6FCF
:103CB000636174696F6E5F726573706F6E73652890
:103CC00043616E617264496E7374616E63652A2C20
:103CD0002043616E61726452785472616E736665DE
:103CE000722A290063616E617264496E6974000012
:103CF00063616E6172645365744C6F63616C4E6F87
:103D0000646549440000000063616E61726448614B
:103D10006E646C6552784672616D650063616E61B8
:103D200072644465636F64655363616C6172000023
:103D300063616E617264456E636F64655363616C49
:103D400061720000696E6372656D656E74547261B4
:103D50006E73666572494400656E7175657565546C
:103D6000784672616D65730070757368547851752B
:103D70006575650070726570617265466F724E653B
:103D800078745472616E736665720000636F707947
:103D90004269744172726179000000006465736366
:103DA00061747465725472616E7366657250617984
:103DB0006C6F61640000000066726565426C6F6341
:103DC0006B0000006269745F6C656E677468203E0A
:103DD00020300072656D61696E696E675F6269743B
:103DE00073203E203000696E7075745F6269745F85
:103DF0006F6666736574203E3D20626C6F636B5F17
:103E00006269745F6F666673657400626C6F636B82
:103E10005F656E645F6269745F6F66667365742068
:103E20003E20626C6F636B5F6269745F6F6666737E
:103E300065740072656D61696E696E675F62697451
:103E40005F6C656E677468203C3D2072656D6169CA
:103E50006E696E675F6269747300696E7075745F16
:103E60006269745F6F6666736574203C3D2074728E
:103E7000616E736665722D3E7061796C6F61645F0F
:103E80006C656E202A2038006F75747075745F62DF
:103E900069745F6F6666736574203C3D203634003C
:103EA00072656D61696E696E675F6269745F6C658A
:103EB0006E677468203D3D20300028726573756C14
:103EC00074203E2030292026262028726573756CC8
:103ED00074203C3D20363429202626202872657324
:103EE000756C74203C3D206269745F6C656E67740C
:103EF0006829000064657374696E6174696F6E206F
:103F0000213D202828766F6964202A2930290076EF
:103F1000616C756520213D202828766F6964202A10
:103F2000293029006F66667365745F776974686904
:103F30006E5F626C6F636B203C2028333255202DFE
:103F4000205F5F6275696C74696E5F6F666673652A
:103F5000746F66202843616E61726442756666659F
:103F600072426C6F636B2C206461746129290000BC
:103F70006F75745F696E7320213D202828766F6904
:103F800064202A29302900007372635F6C656E20FB
:103F90003E203055000000002863616E5F69642098
:103FA0002620307831464646464646465529203D2D
:103FB0003D2063616E5F696400000000616C6C6F9E
:103FC0006361746F722D3E73746174697374696395
:103FD000732E63757272656E745F75736167655F6A
:103FE000626C6F636B73203E203000007472616EF0
:103FF000736665725F696420213D202828766F69A9
:1040000064202A293029000073746174652D3E6292
:1040100075666665725F626C6F636B73203D3D20F1
:104020002828766F6964202A293029002E2E2F2E09
:104030002E2F6D6F64756C65732F6C696263616E92
:104040006172642F63616E6172642E6300697465CE
:104050006D2D3E6672616D652E646174615F6C6585
:104060006E203E20300000006D61696E000000008F
:1040700088400008D01A0020801B002001000000AA
:10408000BD3000080000000069646C65000000009D
:104090000C880000887B888888588828800E00005B
:1040A00088181118987B8888000000008888888804
:1040B00088888888040000008882888888888888A2
:1040C00000000000888888888888888800000000B0
:1040D000E1340008CD34000809350008F534000843
:1040E00001350008ED340008D9340008C534000853
:1040F000153500082C2066756E6374696F6E3A2062
:1041000000617373657274696F6E202225732220BB
:104110006661696C65643A2066696C652022257366
:10412000222C206C696E65202564257325730A0096
:1041300090C0FF7F01000000FFFFFFFF6400000050
:1041400000000000FE2A0100D20400001808002030
:10415000000000000000000000000000000000005F
:10416000000000000000000000000000000000004F
:10417000000000000000000000000000000000003F
:10418000000000000000000000000000000000002F
:10419000000000000000000000000000000000001F
:1041A000000000000000000000000000000000000F
:00000001FF
